:100000008AC00000BEC00000BCC00000BAC0000032
:10001000B8C00000B6C00000B4C00000B2C000000C
:10002000B0C00000AEC00000ACC00000CDC40000F5
:10003000A8C00000A6C00000A4C00000A2C000002C
:10004000A0C000009EC00000BEC000009AC000001A
:1000500098C0000096C0000094C0000092C000004C
:1000600090C000008EC000008CC000008AC000005C
:1000700088C0000012011001FF000040501DC86040
:10008000000101020301090212000101008032098E
:1000900004000000FF000000040309044E034800B0
:1000A00065006E006E0069006E006700200042006F
:1000B00065006B0065006C0020003C0068002E00AD
:1000C000620065006B0065006C00400067006F0017
:1000D0006F0067006C0065006D00610069006C00D6
:1000E0002E0063006F006D003E00000024035800E6
:1000F0006C0069006E006B00200055005300420048
:10010000200041006400610070007400650072000E
:1001100000000203000011241FBECFEFD2E0DEBFBB
:10012000CDBF04B603FE0DC0809113019091140160
:10013000A0911501B09116018E5B9A4BAD4EBE4F4A
:1001400001F01092130110921401109215011092F7
:100150001601E0E0F0E3099511E0A0E0B1E0ECEB7E
:10016000FDE002C005900D92A030B107D9F711E073
:10017000A0E0B1E001C01D92A331B107E1F739D28F
:100180001BC63ECFF8941092850010928400109206
:1001900002011092030110920401109205011092C5
:1001A00001011092000178940895F89481E0809301
:1001B0006F001092850010928400E1E8F0E08081E9
:1001C00083608083DFCF1F920F920FB60F921124AE
:1001D0008F939F93AF93BF938091020190910301FE
:1001E000A0910401B09105010196A11DB11D80935C
:1001F000020190930301A0930401B0930501809143
:10020000020190910301A0910401B0910501B695FE
:10021000A795979587959093010180930001BF91D1
:10022000AF919F918F910F900FBE0F901F901895D7
:100230003A9A429A089522982A9A089583B184702E
:100240008093060108953D98459808953D9A4598F4
:1002500008958091E800877F8093E80093B19470BF
:10026000809106018917C1F09093060191E0809179
:10027000E80080FFFCCF9093F1008091E8008E7F32
:100280008093E8008091E80082FFFCCF8091E80035
:100290008B7F8093E800089590E0E9CFCF92DF92C2
:1002A000FF920F931F93CF93DF936C01EB0110919B
:1002B00006018091E800877F8093E800C114D10493
:1002C00041F18091E80082FFFCCFF090F200FF2026
:1002D000B1F000E08091F1008BB94298429A52DF70
:1002E000209791F503C013B11470A8958091060171
:1002F0001817C9F3109306010F5F0F1558F3CF18A5
:10030000D1088091E8008B7F8093E800C114D1046C
:10031000C1F68091E80080FFFCCF8091E8008E7FDD
:100320008093E800DF91CF911F910F91FF90DF90B4
:10033000CF90089513B11470A89580910001909109
:1003400001018C179D0728F480910601181791F37D
:10035000D1CF8091E8008E7F8093E8008091E80003
:1003600080FFD7CFDACFDF92EF92FF920F931F93E8
:10037000CF93DF937C01EB01109106018091E8009F
:10038000877F8093E800E114F10471F18091E80027
:1003900080FFFCCFC70121E4E216F10410F080E4F5
:1003A00090E0D82E8823B1F000E0ECDE2097B9F57C
:1003B00003C013B11470A895809106011817C9F3F2
:1003C0001093060189B18093F1004298429A0F5F21
:1003D0000D1558F3ED18F1088091E8008E7F809399
:1003E000E800E114F10491F68091E80082FFFCCF6F
:1003F0008091E8008B7F8093E800DF91CF911F917F
:100400000F91FF90EF90DF90089513B11470A895AD
:1004100080910001909101018C179D0728F4809133
:100420000601181791F3CCCF8091E8008E7F80935E
:10043000E8008091E80082FFD7CFDACFE8EEF0E065
:100440008081877F808389B18093F10080818E7F56
:1004500080833FC2E8EEF0E09081977F90838BB974
:1004600080818B7F808335C2E8EEF0E08081877FDA
:1004700080838FEF8AB980818B7F80832AC2E8EEE8
:10048000F0E08081877F80831AB88FEF8BB98081FD
:100490008B7F80831EC22EE088E190E00FB6F89437
:1004A000A895809360000FBE2093600080E090E0EC
:1004B00020E80FB6F89420936100809361000FBE8E
:1004C00074DEC1DEB5DEB7DEB9DED9CFE8EEF0E02E
:1004D0008081877F80834298429A80818B7F80834E
:1004E000F8C10F931F9308EE10E0F8018081877F19
:1004F0008083ACDE80E29EE40197F1F7A4DEF80190
:1005000080818B7F8083E5D11F910F910895809129
:10051000E800877F8093E8008091E8008B7F8093DC
:10052000E800D7D1F6D1F89420E030E048EC50E074
:10053000CA010197F1F72F5F3F4F8EE42032380751
:10054000B9F78EEB9AEBADEEBEEF8093130190936B
:100550001401A0931501B09316012CE088E190E0FE
:100560000FB6F894A895809360000FBE20936000AA
:10057000FFCF80910B01282F30E0C9018076907069
:100580008034910509F008952F713070232BD9F72D
:1005900030910D0160910F01709110018091110156
:1005A0009091120120910C012530F9F0263038F499
:1005B000223081F0233078F4213029F792CF28308F
:1005C00041F0293068F4263091F02730E1F6832F8E
:1005D00041CF64CE7BCF233059F02430A1F64FCFEA
:1005E000293021F02A3079F692CF3ECFBCCE26CFEB
:1005F00030CEDBD150DF7894D7D3A895FDCFDA0188
:100600009230F1F0933091F0913041F0E0E0F0E081
:1006100020E030E0ED93FC93C9010895E4E7F0E0B9
:1006200022E130E0ED93FC93C9010895813081F01F
:100630008130A0F4E8E9F0E08491282F30E0EACF9F
:10064000E6E8F0E022E130E0ED93FC93C901089583
:10065000ECE9F0E08491282F30E0DCCF823039F0F3
:100660008330A1F6E2E1F1E022E030E0D3CFECEE1E
:10067000F0E08491282F30E0CDCF9C0180911101D2
:10068000909112018617970708F062C0BC01F9012A
:1006900090E061157105A1F1992309F467C08EB34B
:1006A000882309F45FC0853009F450C08091E800C8
:1006B00083FD5AC08091E80082FD3FC08091E80030
:1006C00080FFEDCF8091F200282F30E00AC08191A9
:1006D0008093F100615070402F5F3F4F61157105AD
:1006E00019F02034310598F390E02034310519F1E8
:1006F0008091E8008E7F8093E8006115710561F6B6
:100700009923D9F08EB3882369F18530F9F080916F
:10071000E80083FD29C08091E80082FD0EC0809131
:10072000E80080FFEFCF8091F200282F30E090E0CA
:1007300020343105E9F691E0DBCF8091E80082FDBD
:1007400027C08EB3882371F08530B9F783E0089510
:100750006115710509F09BCF8091E8008E7F809331
:10076000E80095CF82E0089581E008958EB3882354
:10077000C9F3853059F38091E80083FDF5CF80916E
:10078000E80082FDDACF8091E80080FFEFCF9ACFBA
:1007900080E008959C0180911101909112018617CB
:1007A000970708F063C0BC01F90190E0611571057D
:1007B000A9F1992309F468C08EB3882309F460C0B5
:1007C000853009F451C08091E80083FD5BC08091C1
:1007D000E80082FD40C08091E80080FFEDCF80916D
:1007E000F200282F30E00BC084918093F100319605
:1007F000615070402F5F3F4F6115710519F0203433
:10080000310590F390E02034310519F18091E80032
:100810008E7F8093E8006115710559F69923D9F010
:100820008EB3882369F18530F9F08091E80083FD6B
:1008300029C08091E80082FD0EC08091E80080FF11
:10084000EFCF8091F200282F30E090E02034310586
:10085000E9F691E0DBCF8091E80082FD27C08EB3FE
:10086000882371F08530B9F783E00895611571052B
:1008700009F09ACF8091E8008E7F8093E80094CFB2
:1008800082E0089581E008958EB38823C9F385300E
:1008900059F38091E80083FDF5CF8091E80082FD57
:1008A000DACF8091E80080FFEFCF99CF80E0089504
:1008B0008091EB0081608093EB001092ED006093DB
:1008C000EC004093ED008091EE00881F8827881F80
:1008D000089580910B01882344F08091E80080FD09
:1008E0000CC08EB38823C9F708958091E80082FD7B
:1008F0000AC08EB38823C9F708958091E8008E7FDF
:100900008093E80008958091E8008B7F8093E80051
:10091000089554D056D0E0EEF0E08081816080836D
:10092000E8EDF0E080818F77808319BCE3E6F0E0AA
:1009300080818160808310920A0108953FD041D068
:100940008091D8008F778093D8008091D8008068FC
:100950008093D8008091D8008F7D8093D80019BCF7
:1009600082E089BD09B400FEFDCF1EBA10920701D6
:10097000109209011092080180E060E042E398DFE4
:100980008091E1008E7F8093E1008091E2008160A0
:100990008093E2008091E20088608093E200809181
:1009A000E0008E7F8093E0000895E3E6F0E0808130
:1009B0008E7F808381E080930A01C0CF1092E20095
:1009C00008951092E10008951F920F920FB60F92B2
:1009D00011242F933F934F935F936F937F938F9344
:1009E0009F93AF93BF93EF93FF938091E10082FFBA
:1009F00004C08091E20082FD7BC08091E10080FF15
:100A000004C08091E20080FD60C08091E10084FF1D
:100A100026C08091E20084FF22C019BC82E089BD1B
:100A200009B400FEFDCF8091D8008F7D8093D8005F
:100A30008091E1008F7E8093E1008091E2008F7EC3
:100A40008093E2008091E20081608093E2008091D7
:100A50000701882309F453C084E08EBBA4D18091A0
:100A6000E10083FF21C08091E20083FF1DC08091DF
:100A7000E100877F8093E10082E08EBB1092070146
:100A80008091E1008E7F8093E1008091E2008E7F73
:100A90008093E2008091E20080618093E20080E038
:100AA00060E042E305DF7FD1FF91EF91BF91AF910D
:100AB0009F918F917F916F915F914F913F912F9176
:100AC0000F900FBE0F901F9018958091E2008E7FBF
:100AD0008093E2008091E20080618093E200809147
:100AE000D80080628093D80019BC1EBA5CD18DCF2B
:100AF0008091E1008B7F8093E10055D17ECF809182
:100B0000E30087FD03C081E08EBBA8CF83E08EBBEE
:100B1000A5CF1F93DF93CF93CDB7DEB7AC970FB6BA
:100B2000F894DEBF0FBECDBF8091F10080930B0122
:100B30008091F10080930C018091F10080930D0170
:100B40008091F10080930E018091F10080930F015C
:100B50008091F100809310018091F1008093110148
:100B60008091F1008093120104DD8091E80083FF01
:100B700011C090910B0180910C018530E1F186301C
:100B800008F1883009F4ACC0893009F490C086308F
:100B900009F451C08091E80083FF0AC08091E80009
:100BA000877F8093E8008091EB0080628093EB0068
:100BB000AC960FB6F894DEBF0FBECDBFCF91DF91DC
:100BC0001F910895813029F0813008F459C0833095
:100BD00009F79923F9F690910D019130D9F6109209
:100BE0000901833009F4DCC08091E800877F80939D
:100BF000E8006FDECFCF992369F610910D011F77C2
:100C00008091E3008078812B8093E3008091E8005D
:100C1000877F8093E8005DDE8091E80080FFFCCF55
:100C20008091E30080688093E300112309F06BC09A
:100C300082E08EBBAFCF9058923008F0ABCF80915E
:100C40000D0190910E0123E08C3D920709F467C0DD
:100C500060910F01AE014F5F5F4FD1DCBC01009787
:100C600009F498CF8091E800877F8093E80089811C
:100C70009A8190DD8091E8008B7F8093E8008ACF95
:100C8000903809F443C0923809F084CF90E0809105
:100C9000E800877F8093E8009093F1001092F100C4
:100CA0008091E8008E7F8093E80013DE73CF992354
:100CB00009F070CF90910D01923008F06BCF8091C8
:100CC000E800877F8093E8009093070102DE80911F
:100CD0000701882309F45AC084E08EBB64D05ACF40
:100CE000903809F057CF8091E800877F8093E80023
:100CF000809107018093F1008091E8008E7F8093BE
:100D0000E800E7DD47CF83E08EBB44CF9091080138
:100D100080910901882309F4BACF9260B8CF83E0AB
:100D20008C838AE28B836FB7F894DE0115964EE0D0
:100D300020E030E051E209C090E0C7968D939D938A
:100D40002F5F3F4F2431310581F0E42FF0E05093C5
:100D50005700849120FF03C082958F704F5F8F7082
:100D60008A3050F790E0C096E9CF6FBF8091E800DD
:100D7000877F8093E800CE0103966AE270E07DDC15
:100D80008091E8008B7F8093E80004CF8091E3009E
:100D900087FD03C081E08EBBA1CF84E08EBB9ECFD8
:100DA0009093090121CF08958EB3882319F0809183
:0C0DB000E80083FF0895ADCEF894FFCF5B
:00000001FF
